:1000000012C07BC02AC029C028C027C09EC025C0FE
:1000100024C023C022C0E1C020C01FC01EC01DC01C
:100020001CC01BC01AC011241FBECFE5D4E0DEBF28
:10003000CDBF10E0A0E6B0E0EAEEF2E002C005902D
:100040000D92A036B107D9F712E0A0E6B0E001C0EA
:100050001D92A736B107E1F701C0D2CFCFE5D4E0BA
:10006000DEBFCDBF12D102D07894FFCF21B3237F62
:10007000286021BB1FBC22E02EBD829903C0000076
:10008000829BFDCF829B03C000008299FDCF1DBCE7
:100090001CBC829903C00000829BFDCFACB5BDB5EE
:1000A0006B2F772720E030E0AD01485E5340A8EE8B
:1000B000B3E0E5E6F2E02083318383E0283E3807B1
:1000C00010F4A083B183808191814817590710F4FF
:1000D000408351833297260F371F80E0E736F807B9
:1000E00054F755B75C7F516055BF4BB74F734064B1
:1000F0004BBF39B7306139BF08951F920F920FB6C9
:100100000F9211242F933F938F939F93AF93BF939D
:10011000EF93FF9320916000A22FBB27AA0FBB1F74
:10012000A959BF4F2D913C913BBD2ABD1DBC1CBCA4
:10013000FF91EF91BF91AF919F918F913F912F913F
:100140000F900FBE0F901F9018951F920F920FB631
:100150000F9211242F938F9320916000222309F492
:1001600032C0939A00000000000000000000000070
:10017000000000000000000000000000000000007F
:10018000000000000000000000000000000000006F
:10019000000000000000000000000000000000005F
:1001A000000000000000000000000000000000004F
:1001B000000000000000000000000000000000003F
:1001C0000000000093988F912F910F900FBE0F9019
:1001D0001F9018958093600008951F920F920FB69C
:1001E0000F9211242F933F934F935F936F937F93BD
:1001F0008F939F93AF93BF93EF93FF938BB14CB1CA
:10020000992784FF03C0109261002EC09C012870C2
:10021000307083FF04C08FEF8093610025C0809110
:100220006100882351F44423B9F741E04093610011
:10023000309363002093620017C08130A9F4A0912D
:100240006200B0916300BD011196B0936300A0936A
:10025000620083B39927809590958F73907068178B
:10026000790711F4842FB6DFFF91EF91BF91AF9121
:100270009F918F917F916F915F914F913F912F91BE
:100280000F900FBE0F901F90189564B3607C64BBF5
:1002900055B35F6355BB949841B34C7E426141BBFB
:1002A00010BC33E039B91BB820E92AB92EE820BDCB
:1002B0000895E199FECF9FBB8EBB6DBBE29AE19A98
:1002C00008959C01872F9927E199FECF3FBB2EBB54
:1002D0008DBBE29AE19AC9010196E199FECF9FBBDD
:0A02E0008EBB6DBBE29AE19A08950F
:00000001FF
